:020000040000FA
:020000000528D1
:0800080009009101830185014B
:10001000860181010301831686011F30850083302C
:10002000810083128B016400051A1328050819202A
:100030001328820789282A282A282A282A282A28B1
:100040002A282A282A282A2877282A282A282A28D3
:100050008F289128932094000A309200F730930063
:100060001409950064002030910086146E208610DB
:100070006B20061506116400861462200310950C8F
:10008000940C930C920C031C4828861065204A2877
:1000900086105F20910B3B288614622086100B305F
:1000A00099006B20990B512886146E2086106820C9
:1000B000861462208610051A080064005B28E93067
:1000C00081007228DD3081007228BB3081007228E7
:1000D0008B30810072281A30810072286B206B20CF
:1000E0006520080064000108031D7228080006103E
:1000F0008420842006140A3098008420980B7D28E0
:1001000000302B20843013289A016B209A0B85280D
:10011000080055302B20842055302B20132806143E
:10012000132806101328820755344D3447345434AD
:100130004E344A3442344F344B3418340034003493
:0801400000344C34003400349B
:02400E00F53F7C
:00000001FF
